S123F8000F8690B710398E00FF8630B710308640B710248608B710268602B710098632B792
S123F820102B862CB7102DB6102F7F000B7F000C0ECE08E0C60218CE0019BDF851BDF8771C
S123F840960C2703BDF9AF7EF83DDF09DE0926FC3918DF03BDFAD018DE0318DF0718DE0721
S123F86026FB7F10227F102018DE0318DF0718DE0726FB5A26DE39960B81FF27037EF92A6B
S123F8807F000B7F000CBDFAA896008141273E8161273A81422748816227448143274E81B6
S123F8A063274A8144275881642754815227628172275E8153275E8173275A8130250981CA
S123F8C0372205BDF92B2062BDF94B205DCEFC61BDFAC3F610004FBDFA63BDFAA8204B7F88
S123F8E01004CEFC76BDFAC3BDFAA8203DCEFC68BDFAC3F610034FBDFA63BDFAA8202BCEE4
S123F900FC6FBDFAC3F610084FBDFA63BDFAA82019970C2015CEFC85BDFAC3BDFAA8CE0819
S123F920E0C60218CE0019BDF85139C60180302704584A26FCF510042703532007FA1004BC
S123F940F7100439F41004F7100439BDFAB3CEFC0FBDFAC3BDFAA8CEFBE9BDFAC3BDFAA86C
S123F960CEFC0FBDFAC3BDFAA8CEFB10BDFAC3BDFAA8CEFB29BDFAC3BDFAA8CEFB44BDFA90
S123F980C3BDFAA8CEFB5DBDFAC3BDFAA8CEFB76BDFAC3BDFAA8CEFB99BDFAC3BDFAA8CE21
S123F9A0FBBDBDFAC3BDFAB3CEFBE7BDFAC3398630B71030CEFC39BDFAC3F610314FBDFADD
S123F9C0638620BDFA9FCEFC3EBDFAC3F610324FBDFA638620BDFA9FCEFC43BDFAC3F61018
S123F9E0334FBDFA638620BDFA9FCEFC48BDFAC3F610344FBDFA638620BDFA9F8634B710BF
S123FA0030CEFC4DBDFAC3F610314FBDFA638620BDFA9FCEFC52BDFAC3F610324FBDFA634E
S123FA208620BDFA9FCEFC57BDFAC3F610334FBDFA638620BDFA9FCEFC5CBDFAC3F61034B3
S123FA404FBDFA63860DBDFA9F394FCE0064028FD7018FCE000A02D7028F58585858DA0220
S123FA60D702394FBDFA4A96018B30BDFA9F9602BDFA74393684F044444444810A2D068084
S123FA800A8B4120028B30BDFA9F3236840F810A2D06800A8B4120028B30BDFA9F3239F6B6
S123FAA0102E2AFBB7102F39860DBDFA9F860ABDFA9F39860DBDFA9F860ABDFA9F860ABD8C
S123FAC0FA9F39A60081FF2706BDFA9F0820F4390FDF058640B71020B71023B710220E3998
S123FAE0DE07270309DF07DE09270309DF098640B710253BB6102EB6102F970086FF970B6E
S123FB003BDC05F31018FD1018CE10001D23BF3B4120203D3E2053484F5720504F5254208B
S123FB204120535441545553FF4220203D3E20434C45415220504F52542042204F555450CA
S123FB40555453FF4320203D3E2053484F5720504F5254204320535441545553FF442020F8
S123FB603D3E2053484F5720504F5254204420535441545553FF5220203D3E2053484F576B
S123FB80205245414C2D54494D4520414E414C4F472056414C554553FF5320203D3E204290
S123FBA045455020535045414B45522028434F4E4E45435420544F2050413629FF30205474
S123FBC04F2037203D3E20544F47474C45205448452053454C4543544544204220504F5221
S123FBE054204C494E45FF3FFF20202041444150542D31312044454D4F2050524F4752419F
S123FC004D20434F4D4D414E44204D454E55FF5F5F5F5F5F5F5F5F5F5F5F5F5F5F5F5F5FD1
S123FC205F5F5F5F5F5F5F5F5F5F5F5F5F5F5F5F5F5F5F5F5F5F5F5FFF4144303DFF414463
S123FC40313DFF4144323DFF4144333DFF4144343DFF4144353DFF4144363DFF4144373D71
S123FC60FF504F5254413DFF504F5254433DFF504F5254443DFF504F5254204220434C459B
S116FC8041524544FF3E3E3E204245455021203C3C3CFF68
S123FFD6FAF4F800F800F800F800F800F800F800FB01F800F800F800F800FAE0F800F800AB
S10DFFF6F800F800F800F800F80025
S9030000FC
